:020000040800F2
:10A00000C8D3002061A1000839C2000855B8000873
:10A01000B1C100085DA30008DDD200080000000007
:10A02000000000000000000000000000B5CE0008A5
:10A0300045AA000800000000A5CA0008F5D00008E5
:10A04000C1A10008C1A10008B1D20008B5C600082E
:10A050001DC70008A1AD0008C1A10008C9A90008DA
:10A06000C1A10008C1A10008C1A10008C1A1000848
:10A0700011C30008C1A1000869C60008C1A10008F9
:10A08000C1A10008C1A10008C1A10008C1A1000828
:10A09000C1A10008C1A10008C1A10008C1A1000818
:10A0A000D9D20008C1A10008C1A10008C1A10008BF
:10A0B000C1A10008C1A10008C1A10008C1A10008F8
:10A0C000C1A1000819CB0008C1A10008C1A1000866
:10A0D000C1A1000855C700085DC7000865C7000892
:10A0E0006DC70008E9AD000805AE0008C1A1000871
:10A0F00021AE0008C1A100083DAE000859AE00081D
:10A1000075AE000891AE0008B9AE0008E1AE0008D7
:10A1100009AF000831AF000859AF000881AF00084F
:10A12000A9AF0008C1A10008C1A100089FB800089C
:10A13000A7B8000839CB0008C1A10008C1A10008D8
:10A14000DFF810D000F0BEF80048004781DA0008C0
:10A15000AFF30080C8D3002080F308887047000068
:10A16000184880474FF080404FF04021C8654000BC
:10A17000C8654010C8650846C06D40F48000C865D9
:10A1800011484FF0402148654FF04021C86D20F044
:10A190004040C8650D4880474FF00E000C494FF015
:10A1A00000000C4908800C4880470C480047FEE737
:10A1B000FEE7FEE7FEE7FEE7FEE7FEE7FEE7FEE777
:10A1C000FEE7000001C100080010008121BB00086B
:10A1D000005000400060004021D2000841A100086A
:10A1E0002DE9F05F0546002092469B4688460646CC
:10A1F000814640241BE0284641464746224600F05F
:10A2000050F853465A46C01A914110D31146184689
:10A21000224600F037F82D1A67EB01084F46224618
:10A220000120002100F02EF817EB00094E41201EFE
:10A23000A4F10104DFDC484631462A464346BDE826
:10A24000F09F10B5441A0346944209D28418114471
:10A2500003E011F8013D04F8013D521EF9D210BD92
:10A2600040EA0104A40703D009E010C9121F10C37B
:10A27000042AFAD203E011F8014B03F8014B521EF5
:10A28000F9D210BD202A04DB203A00FA02F10020A6
:10A2900070479140C2F1200320FA03F31943904024
:10A2A0007047202A04DB203A21FA02F0002170478F
:10A2B00021FA02F3D040C2F120029140084319462E
:10A2C00070470000064C074D06E0E06840F00103CF
:10A2D00094E8070098471034AC42F6D3FFF734FFF8
:10A2E00078E0000898E0000810B504466068064968
:10A2F00008602068FFF730FF0A2000F0B9FB024831
:10A300000068804710BD00001400002070B50446AE
:10A310000D46E1B25A2001F031FD21125B2001F01F
:10A320002DFDE9B25C2001F029FD29125D2001F02C
:10A3300025FD70BD70B504460D46E1B2562001F012
:10A340001DFD2112572001F019FDE9B2582001F03E
:10A3500015FD2912592001F011FD70BD10B503A0A3
:10A3600002F0F8FF02F035FE10BD00007761726E5A
:10A37000696E67A3BB4275734661756C7420486152
:10A380006E646C65720D0A004FF04021096A41F05D
:10A3900001014FF04022116200BF4FF04021096AD5
:10A3A00001F48071B1F5807FF7D14FF04021496A07
:10A3B00021F003014FF0402251621146496A516277
:10A3C00000BF4FF04021496A01F48071B1F5807FF0
:10A3D000F7D15249524A1160032806D1111F09686A
:10A3E00041F08041121F116007E04D49091F0968C3
:10A3F00021F080414A4A121F11604FF4C601484AB9
:10A40000121D11604FF4B20111604FF40C11116074
:10A410004FF4580111601160D1064FF04022D16510
:10A420004900D1654910D1655101D16560B93D49F7
:10A43000096801F07F41B1F1124F37D139490968FC
:10A4400021F07F41916631E0022810D13549083171
:10A45000096801F07F41B1F1124F27D1314908312C
:10A46000096821F07F414FF0402291661EE00328E9
:10A470000CD12C49FC3109682B4A914216D129494B
:10A48000F83109684FF0402291660FE02549091D17
:10A49000096801F07F41B1F1124F07D12149091D2F
:10A4A000096821F07F414FF04022916600211C4A4B
:10A4B000121D11601A49091F096821F08041184ACC
:10A4C000121F116015493039121D11604FF04021E3
:10A4D000096A41F008014FF04022116200BF4FF0BD
:10A4E0004021096A01F40061B1F5006FF7D14FF026
:10A4F0004021496A21F003014FF040225162114688
:10A50000496A41F00101516200BF4FF04021496AA0
:10A5100001F40071B1F5007FF7D170473099D8D8B8
:10A5200004380040C00020083598746770B50246B2
:10A530000B46274D2D6845F08045254E3560351D6D
:10A540002D78244E45EA0604224D3035204E361D26
:10A550003560214D2D6845F2AA56B5421DD14FF008
:10A560004025296B53B102F004051DB1114321F0C0
:10A5700004010DE0114381F0040109E002F004053B
:10A580001DB1914341F0040102E0914381F00401C7
:10A590004FF0402529635A2010E03BB14FF0402591
:10A5A0002D6B15434FF04026356306E04FF04025F4
:10A5B0002D6B95434FF040263563FF20044D2D1D34
:10A5C0002C602D1F2D6825F08045014E356070BD33
:10A5D000003800400099D8D8A400200870B504467F
:10A5E0000D46072000F094FA34B1012C2AD0022C39
:10A5F00050D0032C76D176E04FF04020006A40F036
:10A6000001004FF04021086200BF4FF04020006A77
:10A6100000F48070B0F5807FF7D14FF04020406AA1
:10A6200020F003004FF0402148620846406A48622B
:10A6300000BF4FF04020406A00F48070B0F5807F8A
:10A64000F7D179E04FF04020006A40F008004FF069
:10A650004021086200BF4FF04020006A00F4006013
:10A66000B0F5006FF7D14FF04020406A20F00300B2
:10A670004FF0402148620846406A40F001004862BD
:10A6800000BF4FF04020406A00F40070B0F5007F3A
:10A69000F7D151E04FF04020006A40F004004FF045
:10A6A0004021086200BF4FF04020006A00F4806043
:10A6B000B0F5806FF7D14FF04020406A20F00300E2
:10A6C0004FF0402148620846406A40F0020048626C
:10A6D00000BF4FF04020406A00F48060B0F5806F0A
:10A6E000F7D129E027E04FF04020006A40F0100049
:10A6F0004FF04021086200BF4FF04020006A00F494
:10A700008050B0F5805FF7D14FF04020406A20F0D4
:10A7100003004FF0402148620846406A40F00300C1
:10A72000486200BF4FF04020406A00F40060B0F57E
:10A73000006FF7D100E000BF00BF284603F078F8B3
:10A7400070BD00B5034600F01EF84FF04020C06D0C
:10A7500040F400004FF04021C865102B05D1084699
:10A76000006D40F4004008650CE04FF04020006DA3
:10A7700020F400404FF0402108650846006D63F367
:10A780000300086500BD4FF04021C96D21F0404035
:10A790004FF04021C86540F080414FF04022D16524
:10A7A00040F00041D16540F04041D165704770B53F
:10A7B00002460B46002114461D46002002E0265C9E
:10A7C0003144401CA842FADB0846CE1701EB16665E
:10A7D0003612A1EB0621C8B270BD10B50446E1B235
:10A7E000502001F0CBFAC4F30721512001F0C6FA42
:10A7F000C4F30741522001F0C1FA210E532001F0A9
:10A80000BDFA10BD10B50446E1B2542001F0B6FA0D
:10A810002112552001F0B2FA10BD10B500BF01F0B1
:10A82000B7FA00F008000028F9D110BD10B500BF3C
:10A8300001F0AEFA00F008010029F9D110BD10B501
:10A8400000BF01F0A5FA00F004010029F9D010BD05
:10A8500030B530B9534C646A24F47F44514D6C6276
:10A860001AE001280BD14F4C646A24F47F444D4D0B
:10A870006C622C46646A44F42A446C620CE0022840
:10A880000AD1484C646A24F47F44464D6C622C46DD
:10A89000646A44F47F446C6232B9424C246A24F402
:10A8A0004034404D2C621AE0012A0BD13D4C246A01
:10A8B00024F440343B4D2C622C46246A44F400348A
:10A8C0002C620CE0022A0AD1364C246A24F440346B
:10A8D000344D2C622C46246A44F440342C6233B943
:10A8E000304C646A24F47F042E4D6C621AE0012B14
:10A8F0000BD12C4C646A24F47F042A4D6C622C46E4
:10A90000646A44F42A046C620CE0022B0AD1254CE0
:10A91000646A24F47F04234D6C622C46646A44F418
:10A920007F046C6231B91F4C646A24F0FF041D4D32
:10A930006C6222E001290FD11B4C1A4D80352C602E
:10A94000184C646A24F0FF04164D6C622C46646A4D
:10A9500044F0AA046C6210E002290ED1124C114D91
:10A9600080352C600F4C646A24F0FF040D4D6C623E
:10A970002C46646A44F0FF046C620A4C246844F07C
:10A980000544084D2C6000BF064C246804F00044C8
:10A99000B4F1004FF8D0034C246844F00104014D99
:10A9A0002C6030BD00500540FFFF1F0010B5132084
:10A9B00001F000F901F00FF9C4B204F0DF04204601
:10A9C00001F01CF910BD00001C480068806A1B489B
:10A9D0000068806C00F00F0060B118480068806C5F
:10A9E00000F00F001649086008460068134909681E
:10A9F000C1F8980011480068806A104909688867A2
:10AA00000E480068006B0D490968C1F880000B48CA
:10AA10000068806B09490968C1F888000748006828
:10AA2000006C06490968C1F8900004480068806C11
:10AA300002490968C1F8980070470000E80000204A
:10AA4000F000002010B503A002F084FC02F0C1FA6F
:10AA500010BD00007761726E696E67A3BB446562CA
:10AA600075674D6F6E2048616E646C65720D0A00EB
:10AA700001B581B000200A49096841F27072B1FB4A
:10AA8000F2F1009105E000E0401C00998842FBD300
:10AA9000002001994A1E01920029F4D10CBD00004A
:10AAA000CC00002010B5CD2001F084F801F093F81F
:10AAB000C4B204F07F04204601F0A0F810BD10B528
:10AAC000122001F077F801F086F8C4B244F0400497
:10AAD000204601F093F810BD10B50121002000F0D0
:10AAE00037F910BD10B50446204600F0AFF810BD90
:10AAF00010B50446204600F0FDF808B1002010BD56
:10AB00000120FCE710B50121084600F021F910BD35
:10AB10000146054A106820F00F0001F00F021043B3
:10AB2000014A1060704700000038004070B50646CA
:10AB30000C46154622462946304600F0B7F808B1C3
:10AB4000002070BD0120FCE710B50346002002E0A4
:10AB50001C5C0C54401C9042FAD310BD2DE9F84FF8
:10AB600081468A4614464D46D04600BF2146484697
:10AB700000F040FD10B90020BDE8F88FC5F30806CD
:10AB8000C6F500772819C0F3080B26B3AD1B4FF4A8
:10AB9000007229462C48FFF754FBBC4208D92A49C9
:10ABA00088193A464146FFF74CFBE41BB84406E0DF
:10ABB0002549881922464146FFF743FB00242846D1
:10ABC000FFF796FF009080221F492846FFF7AEFF4F
:10ABD000009005F500752FE0B4F5007F16D34FF413
:10ABE000007241461848FFF72CFB2846FFF780FF0C
:10ABF0000090802214492846FFF798FF009005F541
:10AC0000007508F50078A4F5007415E04FF40072A3
:10AC100029460D48FFF715FB224641460A48FFF733
:10AC200010FB2846FFF764FF009080220649284663
:10AC3000FFF77CFF00900024002CCDD1009808B9CC
:10AC4000012099E7002097E7B081002070B5044605
:10AC500010481149086011484860801F88600F48FB
:10AC60002E38086108460168204688471F2002F0F8
:10AC700073FE322060430A49B0FBF1F0451C022DFF
:10AC800000D2022505F00F0002F058FE05480649E3
:10AC9000086070BD515C0004B0830020FB5A0004C2
:10ACA00040420F0003AC8697043800402DE9F04184
:10ACB00004460D46164615B90320BDE8F08104F0A0
:10ACC000030008B10220F8E7B4F1006F04D304EBED
:10ACD00085000649884201D90220EEE70448012395
:10ACE0003246294607692046B847E6E7FFEF0708DE
:10ACF000B083002070B50446C4F3080008B10220F8
:10AD000070BDB4F1006F02D30D48844201D9022016
:10AD1000F6E70C48012182682046904705460A481C
:10AD2000006800F0010040B124F00F0007490860FE
:10AD300040F201200449C1F884012846E0E7000000
:10AD4000FFEF0708B0830020005005408051054008
:10AD5000012800DD7047012900DDFBE7012805D14E
:10AD6000012903D10C4A0D4B1A6013E0012805D1CB
:10AD700021B9094A521E094B1A600BE030B901296A
:10AD800004D1054A921E054B1A6003E0024AD21E06
:10AD9000024B1A6000BFDDE703AC86970438004021
:10ADA0000E48406800F0020040B101200C490870D4
:10ADB0000A48406840F00200084948600748406C73
:10ADC00000F0020040B10120064908700348406CC1
:10ADD00040F00200014948647047000000A00040B4
:10ADE000F4000020F500002010B50021034800F019
:10ADF0005FFA0021024800F05BFA10BD00900140AC
:10AE00000040024010B50121034800F051FA012131
:10AE1000024800F04DFA10BD009001400040024091
:10AE200010B50321034800F043FA0321024800F063
:10AE30003FFA10BD009001400040024010B50521CE
:10AE4000034800F035FA0521024800F031FA10BD40
:10AE5000009001400040024010B50621034800F078
:10AE600027FA0621024800F023FA10BD00900140A5
:10AE70000040024010B50721034800F019FA0721ED
:10AE8000024800F015FA10BD009001400040024059
:10AE900010B50021054800F00BFA0021044800F02D
:10AEA00007FA0021034800F003FA10BD00A001409A
:10AEB000005002400060024010B50121054800F03A
:10AEC000F7F90121044800F0F3F90121034800F0EB
:10AED000EFF910BD00A001400050024000600240A8
:10AEE00010B50221054800F0E3F90221044800F002
:10AEF000DFF90221034800F0DBF910BD00A001409A
:10AF0000005002400060024010B50321054800F0E7
:10AF1000CFF90321044800F0CBF90321034800F0E6
:10AF2000C7F910BD00A0014000500240006002407F
:10AF300010B50421054800F0BBF90421044800F0D5
:10AF4000B7F90421034800F0B3F910BD00A0014097
:10AF5000005002400060024010B50521054800F095
:10AF6000A7F90521044800F0A3F90521034800F0E2
:10AF70009FF910BD00A00140005002400060024057
:10AF800010B50621054800F093F90621044800F0A9
:10AF90008FF90621034800F08BF910BD00A0014095
:10AFA000005002400060024010B50721054800F043
:10AFB0007FF90721044800F07BF90721034800F0DE
:10AFC00077F910BD00A0014000500240006002402F
:10AFD00070B504460D46002C4DD0012C4BD0022CF0
:10AFE00049D0032C47D0042C45D0052C43D0062C47
:10AFF00041D0072C3FD0082C3DD0092C3BD00A2C47
:10B0000039D00B2C37D00C2C35D00D2C33D00E2C46
:10B0100031D00F2C2FD0102C2DD0112C2BD0122C46
:10B0200029D0132C27D0142C25D0152C23D0162C46
:10B0300021D0172C1FD0182C1DD0192C1BD01A2C46
:10B0400019D01B2C17D01C2C15D01D2C13D01E2C46
:10B0500011D01F2C0FD0202C0DD0212C0BD0222C46
:10B0600009D0232C07D0242C05D0252C03D0262C46
:10B0700001D0272C00D103E0B02181A002F0B6FB63
:10B080000DB1012D00D103E0B1217DA002F0AEFB96
:10B09000272C02DD4FF0FF3070BD092C09DB0B2C93
:10B0A00007DC4FF08040C06940F001004FF0804164
:10B0B000C8610E2C09DB0F2C07DC4FF08040C06903
:10B0C00020F002004FF08041C861262C09DB272CBC
:10B0D00007DC4FF08040C06940F004004FF0804131
:10B0E000C861062C09DB072C07DC4FF08040C069E3
:10B0F00020F010004FF08041C861202C09DB252C86
:10B1000007DC4FF08040C06940F080004FF0804184
:10B11000C8611A2C09DB1F2C07DC4FF08040C06986
:10B1200040F480504FF08041C861162C0EDB192C82
:10B130000CDC4FF08040406C20F070404FF08041BC
:10B1400048640846C06940F40050C861122C09DB0D
:10B15000152C07DC4FF08040C06940F480404FF070
:10B160008041C861102C09DB112C07DC4FF08040B6
:10B17000C06940F400404FF08041C861A5BBE010B9
:10B1800040B94648C078224601219140884343494E
:10B19000C87072E00120B0EBE40F09D14048C078DC
:10B1A000A4F1080101228A4090433D49C87064E03F
:10B1B0000220B0EBE40F09D13A48C078A4F11001A5
:10B1C00001228A4090433749C87056E00320B0EB13
:10B1D000E40F0AD13448C078A4F1180101228A4052
:10B1E00090433149C87048E009E03048C078A4F184
:10B1F000200101228A4090432C49C8703DE0E010B4
:10B2000040B92648C078224601219140084323498D
:10B21000C87032E00120B0EBE40F09D12048C078BB
:10B22000A4F1080101228A4010431D49C87024E09E
:10B230000220B0EBE40F09D11A48C078A4F1100144
:10B2400001228A4010431749C87016E00320B0EB72
:10B25000E40F09D11448C078A4F1180101228A40F2
:10B2600010431149C87008E01048C078A4F12001CB
:10B2700001228A4010430D49C87000200CE70000ED
:10B280004D43555F6472765C6472765C7372635C86
:10B2900065706F72745F6472762E63000090014077
:10B2A00000A0014000400240005002400060024007
:10B2B00070B504460D46E67931461BA002F04AF807
:10B2C0000120A840304000282CD0E0790121A9407D
:10B2D0000843E0712048844204D12A4600211FA07F
:10B2E00002F038F82648844204D12A4601211BA0E6
:10B2F00002F030F82348844204D12A46022117A0E4
:10B3000002F028F82048844204D12A46032113A0E1
:10B3100002F020F81D48844204D12A4604210FA0DF
:10B3200002F018F870BD0000656E746572206570DB
:10B330006F727420696E746572727570742E6375A5
:10B340007272656E7420737461747573203D20256C
:10B350003032780D0A00000000900140456E74659F
:10B36000722045504F5254256420696E7465727284
:10B370007570742E50494E203D2025640D0A000042
:10B3800000A0014000400240005002400060024026
:10B3900070B504460D46002C4DD0012C4BD0022C2C
:10B3A00049D0032C47D0042C45D0052C43D0062C83
:10B3B00041D0072C3FD0082C3DD0092C3BD00A2C83
:10B3C00039D00B2C37D00C2C35D00D2C33D00E2C83
:10B3D00031D00F2C2FD0102C2DD0112C2BD0122C83
:10B3E00029D0132C27D0142C25D0152C23D0162C83
:10B3F00021D0172C1FD0182C1DD0192C1BD01A2C83
:10B4000019D01B2C17D01C2C15D01D2C13D01E2C82
:10B4100011D01F2C0FD0202C0DD0212C0BD0222C82
:10B4200009D0232C07D0242C05D0252C03D0262C82
:10B4300001D0272C00D104E040F223115AA002F0E1
:10B44000D5F90DB1012D00D104E04FF4927156A051
:10B4500002F0CCF9272C00DD70BDE010D8B95948B6
:10B46000C07822460121914008435649C870012DF9
:10B4700008D10846407922460121914008435149AC
:10B4800048718FE04F48407922460121914088431E
:10B490004C49487186E00120B0EBE40F1ED14A48C8
:10B4A000C078A4F1080101228A4010434649C870BF
:10B4B000012D09D108464079A4F1080101228A40F2
:10B4C0001043414948716DE03F484079A4F10801BB
:10B4D00001228A4090433C49487163E00220B0EB6E
:10B4E000E40F1ED13948C078A4F1100101228A402E
:10B4F00010433649C870012D09D108464079A4F19E
:10B50000100101228A401043304948714AE02F4817
:10B510004079A4F1100101228A4090432B494871DF
:10B5200040E00320B0EBE40F1ED12948C078A4F11D
:10B53000180101228A4010432549C870012D09D104
:10B5400008464079A4F1180101228A40104320499D
:10B55000487127E01E484079A4F1180101228A4071
:10B5600090431B4948711DE01A48C078A4F120019E
:10B5700001228A4010431749C870012D09D108469D
:10B580004079A4F1200101228A40104311494871F9
:10B5900008E010484079A4F1200101228A4090433C
:10B5A0000C49487100BF57E74D43555F6472765CA4
:10B5B0006472765C7372635C65706F72745F6472E0
:10B5C000762E63000090014000A001400040024040
:10B5D000005002400060024010B5CD2000F0EAFAB1
:10B5E00000F0F9FAC4B244F08004204600F006FBF3
:10B5F00010BD0000024602F0030008B100207047B1
:10B60000B2F1006F03D35018034B984201D90020C8
:10B61000F5E70120F3E7000000F0070810B5CD20A2
:10B6200000F0C8FA00F0D7FAC4B204F0BF04204614
:10B6300000F0E4FA10BD10B5CD2000F0BBFA00F028
:10B64000CAFAC4B244F04004204600F0D7FA10BD54
:10B6500010B5CD2000F0AEFA00F0BDFAC4B204F08F
:10B66000FD0404F0FE04204600F0C8FA10BD10B539
:10B67000CD2000F09FFA00F0AEFAC4B204F0FD0451
:10B6800044F00104204600F0B9FA10BD10B5CD20F9
:10B6900000F090FA00F09FFAC4B244F0020404F003
:10B6A000FE04204600F0AAFA10BD10B5CD2000F02F
:10B6B00081FA00F090FAC4B244F0020444F00104AC
:10B6C000204600F09BFA10BD10B5CC2000F072FAB5
:10B6D00000F081FAC4B204F0DF0444F01004204604
:10B6E00000F08CFA10BD10B5CC2000F063FA00F029
:10B6F00072FAC4B244F0200404F0EF04204600F0D3
:10B700007DFA10BD10B5CC2000F054FA00F063FAB9
:10B71000C4B204F0DF0404F0EF04204600F06EFA37
:10B7200010BD10B5CD2000F045FA00F054FAC4B2B7
:10B7300004F0F70404F0FB04204600F05FFA10BDAB
:10B7400010B5CD2000F036FA00F045FAC4B204F08E
:10B75000F70444F00404204600F050FA10BD10B580
:10B76000CD2000F027FA00F036FAC4B244F0080405
:10B7700004F0FB04204600F041FA10BD10B5CD20C6
:10B7800000F018FA00F027FAC4B244F0080444F0BC
:10B790000404204600F032FA10BD00004FF04020B3
:10B7A000406A00F00302101E06D0012806D00228CD
:10B7B00017D0032819D116E0114918E01148006884
:10B7C00008B911490CE00F480068012801D10F4960
:10B7D00006E00C480068022801D10D4900E00D493F
:10B7E00005E00D4903E00D4901E0002100BF00BF65
:10B7F0004FF040208068C0B2401CB1FBF0F07047B1
:10B8000000127A00D400002000F36F06000E270714
:10B8100080D1F00800688909001C4E0E001BB7009B
:10B8200010B5032000F0C6F900F0D5F9C4B204F059
:10B83000FB04204600F0E2F910BD10B5132000F023
:10B84000B9F900F0C8F9C4B204F07F04204600F052
:10B85000D5F910BD10B503A001F07CFD01F0B9FBD6
:10B8600010BD00007761726E696E67A3BB4861729C
:10B87000644661756C742048616E646C65720D0A73
:10B880000000000010B5012000F094F900F0A3F9C9
:10B89000C4B244F00104204600F0B0F910BD10B568
:10B8A00000F006F810BD10B500F002F810BD000061
:10B8B00008B5002000903C4800793C4908703A489F
:10B8C000C0793B4908700846007800F00100002864
:10B8D00058D13648007800F00400042863D133487A
:10B8E000007800F0020002281ED12F48007900F0F5
:10B8F000010090B12C4840792E4909682E4A1268FF
:10B9000088542D480068401C2B49086026488078E0
:10B9100040F008002449887045E02348807820F0F2
:10B920002000214988703EE02048007800F00100A6
:10B9300008B31E48007800F04000402812D11F488C
:10B9400000681F490968405C174948711C48006835
:10B95000401C1B4908601448807820F020001249E0
:10B96000887020E01048407900909DF80000401C4D
:10B97000C0B2009017E00C48807820F020000A49FF
:10B98000887010E00848807900F0C000401C06492B
:10B9900088710846807940F0010088710846C079B6
:10B9A00040F00100C87108BD00700140F80000209F
:10B9B000F900002008010020FC0000200401002004
:10B9C0000001002030B530B9534C646A24F47F4440
:10B9D000514D6C621AE001280BD14F4C646A24F47B
:10B9E0007F444D4D6C622C46646A44F42A446C6278
:10B9F0000CE002280AD1484C646A24F47F44464D86
:10BA00006C622C46646A44F47F446C6232B9424CE6
:10BA1000246A24F44034404D2C621AE0012A0BD1F0
:10BA20003D4C246A24F440343B4D2C622C46246A5D
:10BA300044F400342C620CE0022A0AD1364C246A09
:10BA400024F44034344D2C622C46246A44F44034AF
:10BA50002C6233B9304C646A24F47F042E4D6C623E
:10BA60001AE0012B0BD12C4C646A24F47F042A4D7C
:10BA70006C622C46646A44F42A046C620CE0022B6B
:10BA80000AD1254C646A24F47F04234D6C622C4651
:10BA9000646A44F47F046C6231B91F4C646A24F018
:10BAA000FF041D4D6C6222E001290FD11B4C1A4D81
:10BAB00080352C60184C646A24F0FF04164D6C62CB
:10BAC0002C46646A44F0AA046C6210E002290ED18C
:10BAD000124C114D80352C600F4C646A24F0FF0429
:10BAE0000D4D6C622C46646A44F0FF046C620A4C93
:10BAF000246844F00544084D2C6000BF064C2468BF
:10BB000004F00044B4F1004FF8D0034C246844F032
:10BB10000104014D2C6030BD00100540FFFF1F00E7
:10BB200010B500214FF08040FEF700FD0121C8074D
:10BB3000FEF7FCFC00214FF00040FEF7F7FC10BDC3
:10BB400010B50246002001B90121052A2FD2DFE8F5
:10BB500002F0030C20262A004FF04023DB6923F07B
:10BB600001034FF04024E36122E04FF04023DB6902
:10BB700043F001034FF04024E3612346DB6823F0E8
:10BB80000F03E3602346DB680B43E3600123A361FB
:10BB90000EE04FF04023DB6803F00F0008E04FF0A9
:10BBA0004023D86C04E04FF04023D96400E000BF8C
:10BBB00000BF10BD10B5044600210C20FFF7E8FBC4
:10BBC000002001F00FF9204601F00CF901210C20B2
:10BBD000FFF7DEFB10BD10B5002400210C20FFF79D
:10BBE000D7FBC02001F0FEF8FF2001F0FBF804466F
:10BBF00001210C20FFF7CCFB204610BD10B50446F8
:10BC000000210C20FFF7C4FB802001F0EBF8204658
:10BC100001F0E8F801210C20FFF7BAFB10BD70B568
:10BC20000446082C06DA1920FFF7C4FF0020FFF7AE
:10BC3000E5FF0CE02046E11704EB5171C910491EE5
:10BC4000CDB21920FFF7B6FF2846FFF7D7FF70BD2A
:10BC500070B50446082C06DA1820FFF7ABFF002069
:10BC6000FFF7CCFF0CE02046E11704EB5171C9103F
:10BC7000491ECDB21820FFF79DFF2846FFF7BEFFF3
:10BC800070BD70B504460D46082C1DDA1420FFF770
:10BC900091FF0020FFF7B2FF1520FFF78BFFE0B206
:10BCA000FFF7ACFF681EC6B21A20FFF783FF3046CD
:10BCB000FFF7A4FF681EC0F307261B20FFF77AFFDB
:10BCC0003046FFF79BFF2BE02046E11704EB517154
:10BCD000C910491ECEB21420FFF76CFF3046FFF7A3
:10BCE0008DFF2046E11704EB5171C910A4EBC1018F
:10BCF000CEB21520FFF75EFF3046FFF77FFF681ECC
:10BD0000C6B21A20FFF756FF3046FFF777FF681ECE
:10BD1000C0F307261B20FFF74DFF3046FFF76EFFED
:10BD200070BD70B50446082C0CDA1620FFF742FFF0
:10BD30000020FFF763FF1720FFF73CFFE0B2FFF79B
:10BD40005DFF1AE02046E11704EB5171C910491E4E
:10BD5000CDB21620FFF72EFF2846FFF74FFF2046F3
:10BD6000E11704EB5171C910A4EBC101CDB217204A
:10BD7000FFF720FF2846FFF741FF70BD70B505466D
:10BD80000C462846FFF716FF2046FFF737FF70BD29
:10BD900010B5002401F07BF80446204610BD70B5B4
:10BDA0000446601EC5B21F20FFF704FF2846FFF7B8
:10BDB00025FF70BD70B50446601EC5B21E20FFF79A
:10BDC000F9FE2846FFF71AFF70BD70B50446601EE5
:10BDD000C5B21C20FFF7EEFE2846FFF70FFF1D201F
:10BDE000FFF7E8FE2812FFF709FF70BD2DE9F041CB
:10BDF00006460F4614461D46DDF818803946304683
:10BE000001F038F92946204601F018F901F05BF9F4
:10BE1000FEF703FDBDE8F08110B50C48C07840F096
:10BE200080000A49C8700846407920F080004871B7
:10BE30006420FEF71DFE0548407940F0800003496C
:10BE400048716420FEF714FE10BD00000090014010
:10BE500010B56420FEF70CFEFFF7DEFF01F0F2F9EB
:10BE60006420FEF705FE00BFFFF792FF00F002001E
:10BE70000028F9D100F038F910BD00002DE9FE4F7F
:10BE80000024464C4648B4FBF0F100FB1140454904
:10BE9000B0FBF1F002900298052804D94048B4FBA9
:10BEA000F0F0441C02E03E48B4FBF0F43E490C7054
:10BEB00004EB84043D490C703D490C700846007841
:10BEC000642801DD6420087038480078642802DDA9
:10BED00064203649087034480078412802DD41204A
:10BEE000314908704FF00308C146C2464FF0050BB8
:10BEF0000521019100912D48007887002C48007899
:10BF000086002948007885000520FFF753FE4FEA98
:10BF1000881141EA4B01C5F3002241EA0200FFF714
:10BF20006DFE0720FFF746FE4FEA8A12009942EAAB
:10BF30004101C7F3002241EA0200FFF75FFE09203A
:10BF4000FFF738FE4FEA8912019942EA4101C6F330
:10BF5000002241EA0200FFF751FE0620FFF72AFE09
:10BF6000E8B2FFF74BFE0820FFF724FEF8B2FFF718
:10BF700045FE0A20FFF71EFEF0B2FFF73FFE00204D
:10BF8000FFF718FE0120FEF773FD8020FFF736FE55
:10BF90000120FEF76DFDBDE8FE8F0000801310024A
:10BFA00040420F00A0860100330000203200002034
:10BFB000310000202DE9F04105460C4616461F468B
:10BFC000DDF8188000F08AFF304601F00EF80CB959
:10BFD00000F093FF012C01D100F09EFF022C01D153
:10BFE00000F0A9FF032C01D100F0B4FF384601F0A6
:10BFF00016F8404601F004F8012D01D101F056F881
:10C000000DB901F06AF8BDE8F08170B50546292147
:10C01000E020FFF7B3FE0321E120FFF7AFFE4FF46E
:10C020007A7090FBF5F041F6846191FBF0F084B2F8
:10C03000A01E84B2E1B2E220FFF7A0FE2112E320AD
:10C04000FFF79CFE0121E420FFF798FEFEF7F7FBC7
:10C050000120FEF70DFD70BD2DE9F04106460C46AE
:10C0600015461F46DDF81880102E01D1FFF74AFB58
:10C07000182E01D1FFF728FB202E01D1FFF733FB4B
:10C08000012C01D1FFF74DFB022C01D1FFF758FB2A
:10C09000032C01D1FFF763FB042C01D1FFF76EFBEA
:10C0A000012D01D1FFF7D4FA022D01D1FFF7DFFAFC
:10C0B000032D01D1FFF7EAFA042D01D1FFF7F5FABC
:10C0C0000FB9FFF7ABFA012F01D1FFF7B4FAB8F1BE
:10C0D000000F01D1FEF7E6FCB8F1010F01D1FFF727
:10C0E0007BFABDE8F081000010B5FFF7C7FE0348FA
:10C0F0000078FFF78AFF00F03CFF10BD32000020FF
:10C1000010B501210C20FEF711FA10BD10B5044640
:10C11000E1B22020FFF732FEC4F307212120FFF710
:10C120002DFEC4F307412220FFF728FE210E232015
:10C13000FFF724FE10BD10B50446E1B22420FFF73E
:10C140001DFE21122520FFF719FE10BD70B5044613
:10C150000D46E1B22620FFF711FE21122720FFF73E
:10C160000DFEE9B22820FFF709FE29122920FFF76A
:10C1700005FE70BD0021002200BF11E0084600222C
:10C1800008E000F001031BB1074B83EA500000E018
:10C190004008521C082AF4D3044B43F82100491CE0
:10C1A000FF29EBD9704700002083B8ED4806002036
:10C1B00010B503A001F0CEF800F00BFF10BD000099
:10C1C0007761726E696E67A3BB4D656D4D616E617F
:10C1D00067652048616E646C65720D0A000000009E
:10C1E00010B50220FFF7E6FCFFF7F5FCC4B204F03F
:10C1F000FB0404F0FD042046FFF700FD10BD10B560
:10C200000320FFF7D7FCFFF7E6FCC4B204F0FD04FF
:10C2100004F0FE042046FFF7F1FC10BD10B55E20CF
:10C22000FFF7C8FCFFF7D7FCC4B204F0FB042046BC
:10C23000FFF7E4FC10BD000010B503A001F08AF880
:10C2400000F0C7FE10BD00007761726E696E67A3D3
:10C25000BB4E4D492048616E646C65720D0A00004A
:10C260002DE9F0410746884614461D46284600F051
:10C2700033F8C5F1030007FA00F60720284100EA69
:10C280000800064306F00706E21704EBD2625211DB
:10C29000920002F1E022D2F800212146E31704EBDC
:10C2A000D3635B11A4EB431C012303FA0CF31A4381
:10C2B0002046E31704EBD3635B119B0003F1E023FB
:10C2C000C3F800210348005D40EA461001490855C3
:10C2D000BDE8F08100E400E00146072323EA010203
:10C2E0001202054B18684FF6FF031840034B184322
:10C2F0001043014B186070470CED00E00000FA0598
:10C300004A0A52020243014B1A60704708ED00E0EE
:10C3100010B57348446C04F0010040B171A001F005
:10C3200019F86F48406C40F001006D49486404F012
:10C330000200022808D170A001F00CF86848406C97
:10C3400040F002006649486404F01000102808D14B
:10C350006EA000F0FFFF6248406C40F010006049A2
:10C36000486404F02000202808D16DA000F0F2FFFE
:10C370005B48406C40F020005949486404F48070E8
:10C38000B0F5807F13D15648806800F48010B0F576
:10C39000801F03D167A000F0DDFF02E06BA000F07A
:10C3A000D9FF4F48406C40F480704D49486404F414
:10C3B0000070B0F5007F08D16AA000F0CBFF4848BC
:10C3C000406C40F400704649486404F48060B0F565
:10C3D000806F13D14248806800F40010B0F5001F50
:10C3E00003D166A000F0B6FF02E06AA000F0B2FF41
:10C3F0003B48406C40F480603949486404F4006074
:10C40000B0F5006F08D169A000F0A4FF3448406C7B
:10C4100040F400603249486404F48050B0F5805F15
:10C4200013D12F48806800F48000B0F5800F03D14D
:10C4300064A000F08FFF02E068A000F08BFF2848A6
:10C44000406C40F480502649486404F40050B0F534
:10C45000005F08D167A000F07DFF2148406C40F4E8
:10C4600000501F49486404F48040B0F5804F13D158
:10C470001B48806800F40000B0F5000F03D163A0F2
:10C4800000F068FF02E067A000F064FF1448406C11
:10C4900040F480401249486404F40040B0F5004F75
:10C4A00008D166A000F056FF0D48406C40F40040F3
:10C4B0000B49486404F48030B0F5803F08D165A092
:10C4C00000F048FF0648406C40F48030044948645E
:10C4D0000348006A634908430149086210BD00002F
:10C4E000004003405043492056445F4C20746F7510
:10C4F0006368210D0A0000005043492056445F48FC
:10C5000020746F756368210D0A00000050434920B4
:10C5100054445F4C20746F756368210D0A0000005D
:10C520005043492054445F4820746F756368210D5F
:10C530000A0000005344494F2064796E616D6963BD
:10C540002D3020746F756368210D0A005344494FE4
:10C55000207374617469632D3020746F7563682172
:10C560000D0A00005344494F207374617469632DB0
:10C570003120746F756368210D0A00005344494FE0
:10C580002064796E616D69632D3120746F75636805
:10C59000210D0A005344494F207374617469632D5F
:10C5A0003220746F756368210D0A00005344494FAF
:10C5B000207374617469632D3320746F756368210F
:10C5C0000D0A00005344494F2064796E616D696320
:10C5D0002D3220746F756368210D0A005344494F52
:10C5E000207374617469632D3420746F75636821DE
:10C5F0000D0A00005344494F207374617469632D20
:10C600003520746F756368210D0A00005344494F4B
:10C610002064796E616D69632D3320746F75636872
:10C62000210D0A005344494F207374617469632DCE
:10C630003620746F756368210D0A00005344494F1A
:10C64000207374617469632D3720746F756368217A
:10C650000D0A00006E7672616D20636C65616E215B
:10C660000D0A000000FFFF000448006840F01F00B2
:10C670004FF04021C1F8900070470000904000400A
:10C6800010B51220FFF796FAFFF7A5FAC4B244F0EE
:10C6900080042046FFF7B2FA10BD10B51220FFF754
:10C6A00089FAFFF798FAC4B204F0F8042046FFF7BD
:10C6B000A5FA10BD1349098821F00101114A118022
:10C6C0001146098841F00401118001210E4A1180B0
:10C6D0000E4A11700E4909780E4A117011460978F8
:10C6E0006C290DD0012004E00949095C094A115464
:10C6F000401C094909888842F6DB0021064A11805E
:10C7000070470000007000403A0000203C0000200C
:10C71000580A002058400020380000200A480088AD
:10C7200040F004000849088008480078401C074988
:10C73000087008460078052804DB002008700120F6
:10C740000349087070470000008000407E00002010
:10C750007C00002000B500F00DF800BD00B500F031
:10C7600009F800BD00B500F005F800BD00B500F007
:10C7700001F800BD00201F4908781E496C3991F866
:10C78000441001F0100141B11A492839097841F0EB
:10C790001001184A6C3A82F8441016492639097873
:10C7A00001F0100139B113492639097841F010021E
:10C7B000104926390A700F492439097801F010010F
:10C7C00041B10C492439097841F01001094A6C3A09
:10C7D00082F8481007492239097801F0100139B16F
:10C7E00004492239097841F01002024922390A70BD
:10C7F000704700006C8001402DE9F04705460E4669
:10C8000014461F46DDE908892DB1012D03D0022D04
:10C8100001D0032D00D103E0252197A000F0E6FF11
:10C82000042C06D02CB1012C03D0022C01D0032CF7
:10C8300000D103E0262190A000F0D8FF35B1012DF2
:10C8400047D0022D7DD0032D7CD1CEE091484069A8
:10C8500040F001008F4948618F48007A20F00100C4
:10C860008D4908720846406820F007004860084675
:10C87000406804F007010843874948600E70084685
:10C88000007A40F0080008720846C0F81080C760BF
:10C8900081486E30007840F001017F486E300170B1
:10C8A000401E007840F001017B486D300170401E51
:10C8B000007840F00100784981F86C000846007A61
:10C8C00040EA890008720846007A40F001000872C8
:10C8D000CFE07048406940F002006E4948616E4800
:10C8E000407A20F001016C484172406820F07000ED
:10C8F000694948600846406804F0070140EA0110B1
:10C90000654948600E700846407A40F00801624868
:10C910004172C0F81C8087615F486E30007840F03B
:10C9200002015D486E300170401E007840F0020147
:10C9300059486D300170401E007840F002005649A1
:10C9400001E00FE094E081F86C000846407A40EA8C
:10C950008900C1B250484172407A40F001014E480E
:10C96000417286E04B48406940F004004949486103
:10C970004948807A20F0010147488172406820F4DC
:10C98000E060454948600846406804F0070140EA15
:10C990000120414948604E7008213F488172C0F82B
:10C9A000288047623C486E30007840F004013A48E5
:10C9B0006E300170401E007840F0040136486D3042
:10C9C0000170401E007840F00400334981F86C008B
:10C9D0000846807A40EA8900C1B22F488172807A85
:10C9E00040F001012C48817243E02A48406940F040
:10C9F0000400284948612848C07A20F001012648EF
:10CA0000C172406820F4E04023494860084640680D
:10CA100004F0070140EA01301F4948604E700821C8
:10CA20001D48C172C0F8348007631B486E3000781F
:10CA300040F0080118486E300170401E007840F048
:10CA4000080115486D300170401E007840F0080064
:10CA5000114981F86C000846C07A40EA8900C1B2E9
:10CA60000D48C172C07A40F001010B48C17200E06C
:10CA700000BF00BFBDE8F0874D43555F6472765C30
:10CA80006472765C7372635C70776D5F6472762E2D
:10CA900063000000001000400080014010B500F06D
:10CAA0007DF910BD10B503A000F054FC00F091FA20
:10CAB00010BD00007761726E696E67A3BB50656E32
:10CAC0006453562048616E646C65720D0A00000064
:10CAD0002DE9F04104460D4617460026E000B0FB64
:10CAE000F5F0401CC0F345000A498872A000B0FB75
:10CAF000F5F08609300A48700E700846807840F0DC
:10CB00002C0088700223202201210846FFF7A8FB91
:10CB1000BDE8F08100300140064840790548407981
:10CB200000F01000102803D102498879487900BF2D
:10CB3000704700000040014010B57348407900F094
:10CB4000200020287BD1704988797049097899B9EB
:10CB5000A5280BD16E490A780978491C6C4B1970CD
:10CB60006C4988540121694A1170CBE00021674A61
:10CB70001170674A1170C5E064490978012913D121
:10CB80005A280BD162490A780978491C604B197000
:10CB90006049885402215D4A1170B3E000215B4A6C
:10CBA00011705B4A1170ADE058490978022913D120
:10CBB00001280BD156490A780978491C544B197041
:10CBC000544988540321514A11709BE000214F4A77
:10CBD00011704F4A117095E04C49097803290BD127
:10CBE0004B490A780978491C494B197049498854BE
:10CBF0000421464A117085E04449097804290BD183
:10CC000043490A780978491C414B197041498854B5
:10CC100005213E4A117075E03C49097805290FD17C
:10CC20003D4908700A783A490B780978491C384C14
:10CC300021703849CA540621344A117062E062E01A
:10CC40003249097806290BD131490A780978491CFB
:10CC50002F4B19702F49885407212C4A117051E02D
:10CC60002A49097807290BD129490A780978491CEA
:10CC7000274B1970274988540821244A117041E034
:10CC800022490978082928D123490978891E89B9B8
:10CC90001F490A780978491C1D4B19701D49885491
:10CCA00000211D4A117001211C4A11700021174AF0
:10CCB000117027E016490A780978491C144B19703D
:10CCC0001449885419460A7813490978891D8A42FB
:10CCD00018DB09210D4A117014E00C490978092963
:10CCE00010D10B490A780978491C094B1970094978
:10CCF00088540021084A11700121084A117000214E
:10CD0000024A117000BF10BD00D00140C4000020D5
:10CD1000C3000020AE800020C600002001000020DB
:10CD20002DE9F04104460D4617460026E000B0FB11
:10CD3000F5F0401CC0F345000A498872A000B0FB22
:10CD4000F5F08609300A48700E700846807840F089
:10CD50002C00887002233D2200210846FFF780FA4C
:10CD6000BDE8F08100D001401CB510208DF8010015
:10CD700000208DF800008DF805008DF804008DF876
:10CD8000030007208DF8020000208DF80600694698
:10CD9000014800F048F81CBD000001401CB500200F
:10CDA0008DF8000010208DF8010007208DF802009A
:10CDB00008208DF8030004208DF8040000208DF871
:10CDC00005008DF806006946054800F02CF80121A1
:10CDD000034800F01DF801210C20FEF7F9F81CBDF6
:10CDE00000100140014600BF0848C08A00F008005A
:10CDF0000028F9D1054A917400BF0448C08A00F0A8
:10CE000001000028F9D10148807C704700100140E2
:10CE100021B1827842F04002827003E0827802F011
:10CE2000BF028270704710B500224FF6FF73C382B5
:10CE300080238371C371427822F00F028B781A43EA
:10CE40004270827800220B79CC7823438C7923437B
:10CE50004C7823431A4382704B78102B0AD14B79BC
:10CE600003700023C3720E238372837B43F0080395
:10CE7000837303E00023C372012383720023C37012
:10CE8000837843F0400383700123C37210BD10B553
:10CE9000002400210C20FEF77BFA4020FFF7A2FFC0
:10CEA000FF20FFF79FFFC4B201210C20FEF770FAAC
:10CEB000204610BD10B503A000F04CFA00F089F830
:10CEC00010BD00007761726E696E67A3BB53564355
:10CED0002048616E646C65720D0A000010B58520F3
:10CEE000FEF768FEFEF777FEC4B244F0080404F0D3
:10CEF000FB042046FEF782FE10BD10B58520FEF72C
:10CF000059FEFEF768FEC4B204F07F0404F0BF04CB
:10CF10002046FEF773FE10BD10B58520FEF74AFED1
:10CF2000FEF759FEC4B204F07F0444F040042046EA
:10CF3000FEF764FE10BD10B58520FEF73BFEFEF740
:10CF40004AFEC4B244F0800404F0BF042046FEF759
:10CF500055FE10BD10B58520FEF72CFEFEF73BFEFA
:10CF6000C4B244F0800444F040042046FEF746FE7C
:10CF700010BD10B5FEF786FCFFF732F9FEF750FC46
:10CF8000FFF73DF9FFF77CFB00F0C0F9FFF785FBE9
:10CF9000FEF753FC00F0C7F9FDF708FD4FF4F07100
:10CFA0004FF44870FEF76DFE8C20FEF7BAFEA0200D
:10CFB000FEF74EFE1420FEF732FE1420FEF705FFAA
:10CFC0000C20FEF7F7FE0320FEF7E9FEFFF726F937
:10CFD00010BD10B5FDF7D7FB4FF04020C06D40F0FD
:10CFE00008004FF04021C86510BD10B50446601E12
:10CFF00084B28420FEF7DEFDE0B2FEF7FFFD10BD37
:10D0000010B504468C20FEF7D5FDE0B2FEF7F6FD24
:10D010008D20FEF7CFFD2012FEF7F0FD10BD10B5FC
:10D0200004468E20FEF7C6FDE0B2FEF7E7FD8F2036
:10D03000FEF7C0FD2012FEF7E1FD10BD70B50446FD
:10D040000D466C20FEF7B6FDE0B2FEF7D7FD6D2071
:10D05000FEF7B0FD2012FEF7D1FD6E20FEF7AAFD0F
:10D06000E8B2FEF7CBFD6F20FEF7A4FD2812FEF715
:10D07000C5FD70BD70B504460D466820FEF79AFDEB
:10D08000E0B2FEF7BBFD6920FEF794FD2012FEF72B
:10D09000B5FD6A20FEF78EFDE8B2FEF7AFFD6B200E
:10D0A000FEF788FD2812FEF7A9FD70BD10B5862099
:10D0B000FEF780FDFEF78FFDC4B244F01004204659
:10D0C000FEF79CFD10BD10B57620FEF773FDE02045
:10D0D000FEF794FDFDF7AAFB10BD10B58620FEF704
:10D0E00069FDFEF778FDC4B204F0EF042046FEF7B8
:10D0F00085FD10BD704700002DE9FF4704460D4631
:10D1000017464FF00009344B0FCB8DE80F00C8468F
:10D110000026032C01DC002C10DAFEF73FFB2F4920
:10D12000086000210220FEF70BFD401C2B49096816
:10D13000B1FBF0F02A490860BDE8FF87FEF72EFB3F
:10D14000804628480460032C01D105B901255DF80B
:10D150002410681CB1FBF0F62348864205D14645F1
:10D160000ED00320FDF7EDFA0AE02048804505D8EF
:10D17000864203D90120FDF7E4FA01E04FF00109EE
:10D180002046FDF701F929460120FDF727FA394627
:10D190000120FEF7D5FCFEF701FB104908600021D5
:10D1A0000220FEF7CDFC401C0C490968B1FBF0F0F1
:10D1B0000B490860094800680C49884203D81020D0
:10D1C000FDF7BFFA05E0B9F1000F02D00120FDF72D
:10D1D000B8FA00BFB0E7000068E00008CC0000200B
:10D1E000D0000020D400002080D1F00800879303F5
:10D1F00010B50A4800F02EFB012200210220FFF7A3
:10D200007BFF00231A4601211846FDF721FB00236E
:10D210001A4601211846FEF7D5FB10BD90D0030039
:10D220000648006840F470000449086004486FF341
:10D2300008000249803908607047000088ED00E06E
:10D2400000A0000870B500240026002500BFFEF7EE
:10D250009FFD00F00200F8B90120FDF709FC012054
:10D26000FEF7A8FC0120FDF703FCFEF7B4FCC6B2F4
:10D2700006F08000802802D1012500240FE0012063
:10D28000FDF7F6FB0120FEF795FC0120FDF7F0FB12
:10D290008020FEF7B3FC02E00025601CC4B225B973
:10D2A000052C02D1FEF7B8FD0024002DCFD070BDB3
:10D2B00000B500F001F800BD0648008840F0080005
:10D2C0000449088000BF0348008800F0800000285F
:10D2D000F9D17047006000407047000010B503A00E
:10D2E00000F038F8FFF775FE10BD00007761726E30
:10D2F000696E67A3BB55736167654661756C742081
:10D3000048616E646C65720D0A00000010B5122051
:10D31000FEF750FCFEF75FFCC4B204F0F7042046B1
:10D32000FEF76CFC10BD10B51320FEF743FCFEF7B2
:10D3300052FCC4B204F0BF042046FEF75FFC10BDEF
:10D3400045F255500249C8804000C880704700002F
:10D35000005000400FB4054B10B503A9044A0298D1
:10D3600000F018F810BC5DF814FB00007DD900082F
:10D370000C01002002E008C8121F08C1002AFAD1DF
:10D3800070477047002001E001C1121F002AFBD145
:10D39000704700002DE9FF4F8DB00F46054600266F
:10D3A00006E025280BD0DDE90F1290476D1C761C96
:10D3B00028780028F5D111B03046BDE8F08F002460
:10D3C000A246A1460122E94900E0044315F8013FC5
:10D3D000203B02FA03F00842F7D128782A2810D01F
:10D3E0006FF02F022878A0F13001092914D80AEB38
:10D3F0008A0102EB410144F0020400EB010A6D1CBA
:10D40000F0E701CF5FEA000A03D544F40054CAF103
:10D41000000A44F002046D1C28782E2817D115F854
:10D42000010F44F004042A280ED06FF02F02287850
:10D43000A0F1300109290AD809EB890102EB410169
:10D4400000EB01096D1CF2E757F8049B6D1C28786E
:10D450006C280FD006DC4C2817D068280DD06A281D
:10D4600014D104E0742810D07A280FD10DE044F4D0
:10D4700000140AE044F4801401E044F44014697894
:10D48000814202D104F580146D1C6D1C28786E2831
:10D490001ED00CDC632830D004DC00288BD0582848
:10D4A00011D19FE0642867D069280CD164E073280B
:10D4B0002DD004DC6F2872D0702804D194E0752838
:10D4C0006ED078286DD0DDE90F129047761C4BE1C5
:10D4D000C4F30250022806D0032809D0042801CF43
:10D4E00009D0066040E101CFF117C0E900613BE1DE
:10D4F00001CF068038E1067036E117F8040B8DF88D
:10D50000000000208DF80100EB46012003E057F8F1
:10D5100004BB4FF0FF3061074FF0000102D40DE073
:10D5200008F10101884649450FDA8045F8DB1BF810
:10D5300008100029F4D108E008F101018846814271
:10D54000FADB1BF808100029F6D1DDE90F23AAEB5E
:10D5500008008146214600F031F9304400EB08060E
:10D5600004E0DDE90F121BF8010B9047B8F1010848
:10D57000F7D221464846F2E00A21C4F302524FF0A6
:10D58000000B0891022A04D001CFC117032A09D049
:10D590000AE0FF1D27F00707F7E8020108E02CE08A
:10D5A0001EE01FE000B2C117042A01D140B2C1172A
:10D5B000021E71F1000206DA0023D0EB030063EBD8
:10D5C00001012D2202E0220504D52B228DF8242012
:10D5D000012203E0E20701D02022F7E7904653E062
:10D5E0000A210BE0102109E010214FF0000B44F05C
:10D5F00004044FF00809089103E008214FF0000BE4
:10D600000891C4F30252022A04D001CF0021032A58
:10D6100006D006E0FF1D27F00707F7E8020103E048
:10D6200080B2042A00D1C0B24FF0000822072BD5E7
:10D630002A78702A07D0DDF820C08CF0100C5CEA44
:10D640000B0C05D00EE040228DF82420012208E0CA
:10D6500050EA010306D030238DF824308DF82520C0
:10D6600002229046089B83F0080353EA0B030BD178
:10D6700050EA010201D1620706D530228DF824203C
:10D680004FF00108A9F101092A78582A04D038A2DC
:10D690000B9208AA0A920BE03AA2F9E75B46089AB5
:10D6A000FCF79EFD0B9B9B5C0A9A521E0A9213701C
:10D6B00050EA0102F2D10A98ADEB000000F1200B14
:10D6C000600702D524F4803401E04FF00109D94508
:10D6D00002DDA9EB0B0000E0002000EB0B01414450
:10D6E0000890AAEB010AE00306D4DDE90F232146E6
:10D6F000504600F063F806444FF0000908E009A91D
:10D7000011F80900DDE90F12904709F10109761CB3
:10D71000C145F4DBE0030CD5DDE90F23214650467B
:10D7200000F04CF8064404E0DDE90F123020904789
:10D73000761C0899481E08900029F5DC08E00A9834
:10D740000A990078491C0A91DDE90F129047761C6E
:10D75000BBF10001ABF1010BF1DC21465046DDE9E4
:10D760000F2300F019F806446D1C21E6092801007A
:10D770003031323334353637383961626364656647
:10D780000000000030313233343536373839414209
:10D7900043444546000000002DE9F04104460025C1
:10D7A0001E461746880404D405E039462020B047B9
:10D7B0006D1C641EF9D52846BDE8F0812DE9F041C5
:10D7C000044600251E469046C80301D5302700E0D8
:10D7D0002027880404D505E041463846B0476D1C33
:10D7E000641EF9D52846BDE8F081000004460D46C8
:10D7F0002A46214602A0FFF7ADFD00BFFEE700006C
:10D8000057726F6E6720706172616D6574657273B7
:10D810002076616C75653A2066696C6520257320F9
:10D820006F6E206C696E652025640D0A0000000093
:10D830004FF04021896821F0FF014FF040229160B4
:10D8400011468968014391601146896941F00201DE
:10D850009161704701B500BF0098411E00910028FA
:10D86000FAD108BD1CB504460020022104231A4643
:10D87000CDE900100120FEF7BFFFFFF70FF9FEF71B
:10D88000E7FA2C48C07840F040002A49C8700846A2
:10D89000407940F040004871012027490870FFF7A7
:10D8A00063FA0020FEF732FC4FF44870FEF743FCA9
:10D8B00000210846FEF74AFC0020FCF78EFF4FF4DB
:10D8C0004870FCF79FFF00210846FCF733FD4FF43A
:10D8D000F0714FF44870FCF719FD5CB14FF6FF7022
:10D8E00040F2DF1340F21F32002100900846FEF79D
:10D8F0007DFA0AE040F21F5040F2DF1340F21F327F
:10D90000002100900846FEF771FA0020034601222C
:10D91000114600901820FEF79FFB4FF4C87043009B
:10D920000522002100900120FEF744FBFDF7C7F817
:10D930001CBD000000900140300000200146054A57
:10D94000106820F00F0001F00F021043014A106030
:10D9500070470000003800400749096821F0F8715D
:10D96000054A11601146096800F01F0241EA0251A0
:10D97000014A1160704700002C38004000BF044A83
:10D98000527902F04002002AF9D0014B9871704799
:10D990000030014070B505460E460024A522214600
:10D9A000641C6A545A222146641C6A54012221468E
:10D9B000641C6A542146641C6E5403222146641C74
:10D9C0006A5400222146641C6A5421462846FCF70A
:10D9D000EEFE2855641C204670BD30B502460B464D
:10D9E0000020A5250446401C15555A250446401C18
:10D9F000155501250446401C15550446401C155577
:10DA000021250446401C155502250446401C155589
:10DA10000446401C155501250146441CE0B25554EE
:10DA200027250146441CE0B2555430BD30B50246AE
:10DA30000B460020A5250446401C15555A250446D2
:10DA4000401C155501250446401C15550446401C34
:10DA5000155521250446401C155502250446401C39
:10DA6000155503250446401C155501250146441C47
:10DA7000E0B2555428250146441CE0B2555430BD4F
:10DA80000021F448FEF73CFCFFF7B2FB62B600222F
:10DA90004FF4E131F0480068FFF71AF800224FF424
:10DAA0001641ED480068FFF73BF9FEF763FBEB48D2
:10DAB000EB490860EBA0FFF74DFC0020FFF7D2FE1A
:10DAC000EEA2F1A1F3A0FFF745FCC1E1FFF738FC9E
:10DAD000F7480068F74988427ED1FFF731FCF648E5
:10DAE0000078012814D10020F3490870F349087028
:10DAF000F3490870F3A0FFF72DFCF6480178F648CB
:10DB0000FFF794FF04462146F34800F07DFA00BF7A
:10DB1000EB4800780128D8D1E8480078401E81B24F
:10DB2000EE48FCF744FE04462246E4480178ECA0A7
:10DB3000FFF710FCE1480078401E81B2E748FCF78F
:10DB400036FEDE490978491EE44A515C884210D00D
:10DB5000DA480078401E81B21046FCF728FE0446E1
:10DB6000D6480078401EDD490A5C2146E1A0FFF757
:10DB7000F1FBDA480078A5280AD0D84840785A281E
:10DB800006D0D6488078012802D0DFA0FFF7E2FB5C
:10DB9000D2480079202832D1D048807901282ED16E
:10DBA000CE48C07901282AD1CC48C078C94908702C
:10DBB00008460178C848FFF7EDFE04460020BF493B
:10DBC0000870BF4908702146C34800F01DFA1E20A6
:10DBD000FCF74EFFBF4800E037E10178BE48FFF791
:10DBE00025FF05460020B5490870B5490870B5A065
:10DBF000FFF7B0FB2946B84800F006FA28E1B7481D
:10DC0000007920287ED1B54880790228FAD1B3481E
:10DC1000C07901287FD1B148407AB049097A4FF4E0
:10DC2000807313FB0102BC480188BCA0FFF792FB84
:10DC3000AA48407AA949097A4FF4807212FB010080
:10DC4000B549098888424DD1A44D0B35A348847A43
:10DC500083480668A148877A32462146B2A0FFF77A
:10DC600079FB32462146284600F0B2F92246B349F4
:10DC70007B480068FCF768FF39462846FCF797FDAB
:10DC8000AF4908703946AD48FCF791FDAD490870C1
:10DC9000AB4800780978884203D1ABA0FFF75AFB64
:10DCA00002E0ABA0FFF756FB6D48006820446C49CA
:10DCB000086099480088401C974908808748C078C8
:10DCC00084490870084601788348FFF763FE804660
:10DCD00000207A4908707A49087041467E4800F071
:10DCE00093F9B5E09CA0FFF735FB7C48C0787949F3
:10DCF0000870084601787848FFF74CFE044600207B
:10DD00006E4900E007E008706D49087021467248CE
:10DD100000F07AF99CE071480079202838D16F48EA
:10DD20008079012834D16D48C079022830D18EA085
:10DD3000FFF710FB6948C07866490870084601780B
:10DD40006548FFF727FE044600205C4908705C49DF
:10DD50000870714908800846018887A0FFF7FAFA21
:10DD600021465D4800F050F95A4801785A48FFF7BB
:10DD700034FE04462146584800F046F900204C493C
:10DD8000086081A0FFF7E6FA3448FCF7ADFA5FE0DF
:10DD90005248007920281ED15048807901281AD194
:10DDA0004E48C079022816D17BA0FFF7D3FA4B4822
:10DDB000C07848490870084601784748FFF7EAFDEF
:10DDC000044600203D4908703D49087021464248FC
:10DDD00000F01AF93CE04148007920281ED13F4864
:10DDE000807901281AD13D48C079022816D16FA048
:10DDF000FFF7B0FA3948C07836490870084601780C
:10DE00003548FFF7C7FD044600202C4908702C490F
:10DE100008702146304800F0F7F819E067A0FFF7D6
:10DE200099FA2E48C0782B490870084601782A488C
:10DE3000FFF7B0FD04460020204908702049087013
:10DE40002146254800F0E0F802E06048FCF74CFA73
:10DE50003CE6000000A00008D000002000000108FF
:10DE60000C0000202A2A2A626F6F746C6F6164654F
:10DE7000723221212A2A0D0A0000000031343A337F
:10DE8000363A3430000000004A756E2020362032C9
:10DE9000303235002064617465203D2025732C7478
:10DEA000696D65203D202573202020200D0A00008B
:10DEB000007003207856341225000020C300002093
:10DEC0000100002073746172742075706461746164
:10DED0000D0A0000C20000209A800020AE800020C1
:10DEE0007265763A256420636865636B3A25780D20
:10DEF0000A000000257820636865636B5F657272B5
:10DF00006F2025780D0A0000696C6C6567616C5F95
:10DF10006E6577210D0A0000C80000202A2A2A25F4
:10DF2000642025640D0A00006C656E3A256420614A
:10DF30006464723A25780D0A00000000190500207B
:10DF40002C0000202D0000202D6F6B0D0A0000001A
:10DF50006661696C0D0A00002A2A2A726570656183
:10DF600074210D0A000000004F54412D66696E694E
:10DF700073680D0A000000006F74615F7365713D86
:10DF800025640D0A000000007475726E20746F2005
:10DF900041505031210D0A004F54412D7265717569
:10DFA0006573742D6661696C0D0A00004F54412D34
:10DFB00074696D656F75740D0A0000006F74686593
:10DFC00072206E6577210D0A0000000000900408A1
:10DFD0002DE9F04104460D4616460A4800684FF404
:10DFE0007A71B0FBF1F73846FCF77CFDFCF78AFD4F
:10DFF0002A4621463046FCF7B1FDFCF76DFD0020B6
:10E00000BDE8F081CC00002070B504460D4611A09B
:10E01000FFF7A0F9002605E0A15D10A0FFF79AF92F
:10E02000701CC6B2AE42F7DB0DA0FFF793F90020DB
:10E030000BE000BF0B49497901F040010029F9D0FC
:10E04000215C084A9171411CC8B2A842F1DB002052
:10E0500070BD000061636B3A00000000202578006D
:10E060000D0A000000D0014000F36F06000E2707E4
:10E0700080D1F0080068890998E0000800000020BD
:10E080001001000074D30008A8E10008100100206E
:10E09000B8D2000084D30008000000000000000097
:10E0A0000000000000000000000000000000000070
:10E0B000000000000000000000000000000100005F
:10E0C000000000000000000001000000000000004F
:10E0D0000000000000000000000000000000000040
:10E0E0000000000000000000000000000000000030
:10E0F0000000000000000000000000000000000020
:10E10000000000000000000000000000000000000F
:10E1100000000000000000000000000000000000FF
:10E120000060044058600440B0600440086104404E
:10E130000070044058700440B070044008710440FE
:10E14000C0620440C07204400000000000000000F3
:10E1500000000000000000000000000000000000BF
:10E1600000000000000000000000000003000000AC
:10E170000060044058600440B060044008610440FE
:10E18000C062044000000000000000000000000029
:10E1900000FF000000000000000000000000000080
:08E1A000000000000000000077
:040000050800A1410D
:00000001FF
